 management

 Timestamp is 389294d4 (reproducible build file hash)

 Preferred load address is 0000000180000000

 Start         Length     Name                   Class
 0001:00000000 000017d0H .text$mn                CODE
 0001:000017d0 00000036H .text$mn$00             CODE
 0001:00001806 00000092H .text$x                 CODE
 0002:00000000 00000138H .idata$5                DATA
 0002:00000138 00000038H .00cfg                  DATA
 0002:00000170 00000008H .CRT$XCA                DATA
 0002:00000178 00000008H .CRT$XCZ                DATA
 0002:00000180 00000008H .CRT$XIA                DATA
 0002:00000188 00000008H .CRT$XIZ                DATA
 0002:00000190 00000008H .CRT$XPA                DATA
 0002:00000198 00000008H .CRT$XPZ                DATA
 0002:000001a0 00000008H .CRT$XTA                DATA
 0002:000001a8 00000008H .CRT$XTZ                DATA
 0002:000001b0 00000000H .gehcont$y              DATA
 0002:000001b0 00000000H .gfids$y                DATA
 0002:000001b0 00000350H .rdata                  DATA
 0002:00000500 00000000H .rdata$CastGuardVftablesA DATA
 0002:00000500 00000000H .rdata$CastGuardVftablesC DATA
 0002:00000500 00000074H .rdata$voltmd           DATA
 0002:00000574 000002bcH .rdata$zzzdbg           DATA
 0002:00000830 00000008H .rtc$IAA                DATA
 0002:00000838 00000008H .rtc$IZZ                DATA
 0002:00000840 00000008H .rtc$TAA                DATA
 0002:00000848 00000008H .rtc$TZZ                DATA
 0002:00000850 000001c0H .xdata                  DATA
 0002:00000a10 0000113cH .edata                  DATA
 0002:00001b4c 00000078H .idata$2                DATA
 0002:00001bc4 00000014H .idata$3                DATA
 0002:00001bd8 00000138H .idata$4                DATA
 0002:00001d10 0000035aH .idata$6                DATA
 0003:00000000 00000080H .data                   DATA
 0003:00000080 00000610H .bss                    DATA
 0004:00000000 0000024cH .pdata                  DATA
 0005:00000000 00000060H .rsrc$01                DATA
 0005:00000060 00000328H .rsrc$02                DATA

  Address         Publics by Value              Rva+Base               Lib:Object

 0000:00000000       __AbsoluteZero             0000000000000000     <absolute>
 0000:00000000       ___safe_se_handler_count   0000000000000000     <absolute>
 0000:00000000       ___safe_se_handler_table   0000000000000000     <absolute>
 0000:00000000       __arm64x_extra_rfe_table   0000000000000000     <absolute>
 0000:00000000       __arm64x_extra_rfe_table_size 0000000000000000     <absolute>
 0000:00000000       __arm64x_native_entrypoint 0000000000000000     <absolute>
 0000:00000000       __arm64x_redirection_metadata 0000000000000000     <absolute>
 0000:00000000       __arm64x_redirection_metadata_count 0000000000000000     <absolute>
 0000:00000000       __dynamic_value_reloc_table 0000000000000000     <absolute>
 0000:00000000       __enclave_config           0000000000000000     <absolute>
 0000:00000000       __guard_check_icall_a64n_fptr 0000000000000000     <absolute>
 0000:00000000       __guard_eh_cont_count      0000000000000000     <absolute>
 0000:00000000       __guard_eh_cont_table      0000000000000000     <absolute>
 0000:00000000       __guard_fids_count         0000000000000000     <absolute>
 0000:00000000       __guard_fids_table         0000000000000000     <absolute>
 0000:00000000       __guard_iat_count          0000000000000000     <absolute>
 0000:00000000       __guard_iat_table          0000000000000000     <absolute>
 0000:00000000       __guard_longjmp_count      0000000000000000     <absolute>
 0000:00000000       __guard_longjmp_table      0000000000000000     <absolute>
 0000:00000000       __hybrid_auxiliary_delayload_iat 0000000000000000     <absolute>
 0000:00000000       __hybrid_auxiliary_delayload_iat_copy 0000000000000000     <absolute>
 0000:00000000       __hybrid_auxiliary_iat     0000000000000000     <absolute>
 0000:00000000       __hybrid_auxiliary_iat_copy 0000000000000000     <absolute>
 0000:00000000       __hybrid_code_map          0000000000000000     <absolute>
 0000:00000000       __hybrid_code_map_count    0000000000000000     <absolute>
 0000:00000000       __hybrid_image_info_bitfield 0000000000000000     <absolute>
 0000:00000000       __x64_code_ranges_to_entry_points 0000000000000000     <absolute>
 0000:00000000       __x64_code_ranges_to_entry_points_count 0000000000000000     <absolute>
 0000:00000100       __guard_flags              0000000000000100     <absolute>
 0000:00000000       __ImageBase                0000000180000000     <linker-defined>
 0001:00000000       Java_sun_management_ClassLoadingImpl_setVerboseClass 0000000180001000 f   ClassLoadingImpl.obj
 0001:00000010       Java_sun_management_GarbageCollectorImpl_getCollectionCount 0000000180001010 f   GarbageCollectorImpl.obj
 0001:00000024       Java_sun_management_GarbageCollectorImpl_getCollectionTime 0000000180001024 f   GarbageCollectorImpl.obj
 0001:00000038       Java_sun_management_HotspotThread_getInternalThreadCount 0000000180001038 f   HotspotThread.obj
 0001:0000004c       Java_sun_management_HotspotThread_getInternalThreadTimes0 000000018000104c f   HotspotThread.obj
 0001:00000060       Java_sun_management_MemoryImpl_getMemoryManagers0 0000000180001060 f   MemoryImpl.obj
 0001:00000070       Java_sun_management_MemoryImpl_getMemoryPools0 0000000180001070 f   MemoryImpl.obj
 0001:00000080       Java_sun_management_MemoryImpl_getMemoryUsage0 0000000180001080 f   MemoryImpl.obj
 0001:00000090       Java_sun_management_MemoryImpl_setVerboseGC 0000000180001090 f   MemoryImpl.obj
 0001:000000a0       Java_sun_management_MemoryManagerImpl_getMemoryPools0 00000001800010a0 f   MemoryManagerImpl.obj
 0001:000000dc       Java_sun_management_MemoryPoolImpl_getCollectionUsage0 00000001800010dc f   MemoryPoolImpl.obj
 0001:000000ec       Java_sun_management_MemoryPoolImpl_getMemoryManagers0 00000001800010ec f   MemoryPoolImpl.obj
 0001:00000128       Java_sun_management_MemoryPoolImpl_getPeakUsage0 0000000180001128 f   MemoryPoolImpl.obj
 0001:00000164       Java_sun_management_MemoryPoolImpl_getUsage0 0000000180001164 f   MemoryPoolImpl.obj
 0001:000001a0       Java_sun_management_MemoryPoolImpl_resetPeakUsage0 00000001800011a0 f   MemoryPoolImpl.obj
 0001:000001b4       Java_sun_management_MemoryPoolImpl_setCollectionThreshold0 00000001800011b4 f   MemoryPoolImpl.obj
 0001:00000224       Java_sun_management_MemoryPoolImpl_setPoolCollectionSensor 0000000180001224 f   MemoryPoolImpl.obj
 0001:0000023c       Java_sun_management_MemoryPoolImpl_setPoolUsageSensor 000000018000123c f   MemoryPoolImpl.obj
 0001:00000254       Java_sun_management_MemoryPoolImpl_setUsageThreshold0 0000000180001254 f   MemoryPoolImpl.obj
 0001:000002c4       Java_sun_management_ThreadImpl_dumpThreads0 00000001800012c4 f   ThreadImpl.obj
 0001:000002e8       Java_sun_management_ThreadImpl_findDeadlockedThreads0 00000001800012e8 f   ThreadImpl.obj
 0001:000002f8       Java_sun_management_ThreadImpl_findMonitorDeadlockedThreads0 00000001800012f8 f   ThreadImpl.obj
 0001:00000308       Java_sun_management_ThreadImpl_getThreadAllocatedMemory0 0000000180001308 f   ThreadImpl.obj
 0001:00000318       Java_sun_management_ThreadImpl_getThreadAllocatedMemory1 0000000180001318 f   ThreadImpl.obj
 0001:0000032c       Java_sun_management_ThreadImpl_getThreadInfo1 000000018000132c f   ThreadImpl.obj
 0001:00000348       Java_sun_management_ThreadImpl_getThreadTotalCpuTime0 0000000180001348 f   ThreadImpl.obj
 0001:0000035c       Java_sun_management_ThreadImpl_getThreadTotalCpuTime1 000000018000135c f   ThreadImpl.obj
 0001:00000378       Java_sun_management_ThreadImpl_getThreadUserCpuTime0 0000000180001378 f   ThreadImpl.obj
 0001:0000038c       Java_sun_management_ThreadImpl_getThreadUserCpuTime1 000000018000138c f   ThreadImpl.obj
 0001:000003a8       Java_sun_management_ThreadImpl_getThreads 00000001800013a8 f   ThreadImpl.obj
 0001:000003b0       Java_sun_management_ThreadImpl_getTotalThreadAllocatedMemory 00000001800013b0 f   ThreadImpl.obj
 0001:000003bc       Java_sun_management_ThreadImpl_resetContentionTimes0 00000001800013bc f   ThreadImpl.obj
 0001:000003d4       Java_sun_management_ThreadImpl_resetPeakThreadCount0 00000001800013d4 f   ThreadImpl.obj
 0001:000003f4       Java_sun_management_ThreadImpl_setThreadAllocatedMemoryEnabled0 00000001800013f4 f   ThreadImpl.obj
 0001:00000404       Java_sun_management_ThreadImpl_setThreadContentionMonitoringEnabled0 0000000180001404 f   ThreadImpl.obj
 0001:00000414       Java_sun_management_ThreadImpl_setThreadCpuTimeEnabled0 0000000180001414 f   ThreadImpl.obj
 0001:00000424       Java_sun_management_VMManagementImpl_getAvailableProcessors 0000000180001424 f   VMManagementImpl.obj
 0001:0000042c       Java_sun_management_VMManagementImpl_getClassInitializationTime 000000018000142c f   VMManagementImpl.obj
 0001:00000440       Java_sun_management_VMManagementImpl_getClassLoadingTime 0000000180001440 f   VMManagementImpl.obj
 0001:00000454       Java_sun_management_VMManagementImpl_getClassVerificationTime 0000000180001454 f   VMManagementImpl.obj
 0001:00000468       Java_sun_management_VMManagementImpl_getDaemonThreadCount 0000000180001468 f   VMManagementImpl.obj
 0001:0000047c       Java_sun_management_VMManagementImpl_getInitializedClassCount 000000018000147c f   VMManagementImpl.obj
 0001:00000490       Java_sun_management_VMManagementImpl_getLiveThreadCount 0000000180001490 f   VMManagementImpl.obj
 0001:000004a4       Java_sun_management_VMManagementImpl_getLoadedClassSize 00000001800014a4 f   VMManagementImpl.obj
 0001:000004b8       Java_sun_management_VMManagementImpl_getMethodDataSize 00000001800014b8 f   VMManagementImpl.obj
 0001:000004cc       Java_sun_management_VMManagementImpl_getPeakThreadCount 00000001800014cc f   VMManagementImpl.obj
 0001:000004e0       Java_sun_management_VMManagementImpl_getProcessId 00000001800014e0 f   VMManagementImpl.obj
 0001:000004f4       Java_sun_management_VMManagementImpl_getSafepointCount 00000001800014f4 f   VMManagementImpl.obj
 0001:00000508       Java_sun_management_VMManagementImpl_getSafepointSyncTime 0000000180001508 f   VMManagementImpl.obj
 0001:0000051c       Java_sun_management_VMManagementImpl_getStartupTime 000000018000151c f   VMManagementImpl.obj
 0001:00000530       Java_sun_management_VMManagementImpl_getTotalApplicationNonStoppedTime 0000000180001530 f   VMManagementImpl.obj
 0001:00000544       Java_sun_management_VMManagementImpl_getTotalClassCount 0000000180001544 f   VMManagementImpl.obj
 0001:00000558       Java_sun_management_VMManagementImpl_getTotalCompileTime 0000000180001558 f   VMManagementImpl.obj
 0001:0000056c       Java_sun_management_VMManagementImpl_getTotalSafepointTime 000000018000156c f   VMManagementImpl.obj
 0001:00000580       Java_sun_management_VMManagementImpl_getTotalThreadCount 0000000180001580 f   VMManagementImpl.obj
 0001:00000594       Java_sun_management_VMManagementImpl_getUnloadedClassCount 0000000180001594 f   VMManagementImpl.obj
 0001:000005a8       Java_sun_management_VMManagementImpl_getUnloadedClassSize 00000001800015a8 f   VMManagementImpl.obj
 0001:000005bc       Java_sun_management_VMManagementImpl_getUptime0 00000001800015bc f   VMManagementImpl.obj
 0001:000005d0       Java_sun_management_VMManagementImpl_getVerboseClass 00000001800015d0 f   VMManagementImpl.obj
 0001:000005e0       Java_sun_management_VMManagementImpl_getVerboseGC 00000001800015e0 f   VMManagementImpl.obj
 0001:000005f0       Java_sun_management_VMManagementImpl_getVersion0 00000001800015f0 f   VMManagementImpl.obj
 0001:0000065c       Java_sun_management_VMManagementImpl_getVmArguments0 000000018000165c f   VMManagementImpl.obj
 0001:00000664       Java_sun_management_VMManagementImpl_initOptionalSupportFields 0000000180001664 f   VMManagementImpl.obj
 0001:000007a0       Java_sun_management_VMManagementImpl_isThreadAllocatedMemoryEnabled 00000001800017a0 f   VMManagementImpl.obj
 0001:000007b0       Java_sun_management_VMManagementImpl_isThreadContentionMonitoringEnabled 00000001800017b0 f   VMManagementImpl.obj
 0001:000007c0       Java_sun_management_VMManagementImpl_isThreadCpuTimeEnabled 00000001800017c0 f   VMManagementImpl.obj
 0001:000007d0       __local_stdio_printf_options 00000001800017d0 f i VMManagementImpl.obj
 0001:0000082c       snprintf                   000000018000182c f i VMManagementImpl.obj
 0001:00000884       JNI_OnLoad                 0000000180001884 f   management.obj
 0001:000008eb       JNU_ThrowInternalError     00000001800018eb f   java:java.dll
 0001:000008f1       JVM_GetAllThreads          00000001800018f1 f   jvm:jvm.dll
 0001:000008f7       JVM_ActiveProcessorCount   00000001800018f7 f   jvm:jvm.dll
 0001:000008fd       JVM_GetVmArguments         00000001800018fd f   jvm:jvm.dll
 0001:00000903       JVM_GetManagement          0000000180001903 f   jvm:jvm.dll
 0001:0000090c       __GSHandlerCheck           000000018000190c f   MSVCRT:gshandler.obj
 0001:0000092c       __GSHandlerCheckCommon     000000018000192c f   MSVCRT:gshandler.obj
 0001:000009a0       __security_check_cookie    00000001800019a0 f   MSVCRT:amdsecgs.obj
 0001:00000cd0       _DllMainCRTStartup         0000000180001cd0 f   MSVCRT:dll_dllmain.obj
 0001:00000d10       __raise_securityfailure    0000000180001d10 f   MSVCRT:gs_report.obj
 0001:00000d44       __report_gsfailure         0000000180001d44 f   MSVCRT:gs_report.obj
 0001:00000e8c       __security_init_cookie     0000000180001e8c f   MSVCRT:gs_support.obj
 0001:00000f38       DllMain                    0000000180001f38 f   MSVCRT:dll_dllmain_stub.obj
 0001:00000f5c       ?__scrt_initialize_type_info@@YAXXZ 0000000180001f5c f   MSVCRT:tncleanup.obj
 0001:00000f6c       ?__scrt_uninitialize_type_info@@YAXXZ 0000000180001f6c f   MSVCRT:tncleanup.obj
 0001:00000f78       __local_stdio_scanf_options 0000000180001f78 f i MSVCRT:default_local_stdio_options.obj
 0001:00000f80       __scrt_initialize_default_local_stdio_options 0000000180001f80 f   MSVCRT:default_local_stdio_options.obj
 0001:00000f9c       __scrt_acquire_startup_lock 0000000180001f9c f   MSVCRT:utility.obj
 0001:00000fd8       __scrt_dllmain_after_initialize_c 0000000180001fd8 f   MSVCRT:utility.obj
 0001:0000100c       __scrt_dllmain_before_initialize_c 000000018000200c f   MSVCRT:utility.obj
 0001:00001024       __scrt_dllmain_crt_thread_attach 0000000180002024 f   MSVCRT:utility.obj
 0001:0000104c       __scrt_dllmain_crt_thread_detach 000000018000204c f   MSVCRT:utility.obj
 0001:00001064       __scrt_dllmain_exception_filter 0000000180002064 f   MSVCRT:utility.obj
 0001:000010c4       __scrt_dllmain_uninitialize_c 00000001800020c4 f   MSVCRT:utility.obj
 0001:000010f4       __scrt_dllmain_uninitialize_critical 00000001800020f4 f   MSVCRT:utility.obj
 0001:00001108       __scrt_initialize_crt      0000000180002108 f   MSVCRT:utility.obj
 0001:00001144       __scrt_initialize_onexit_tables 0000000180002144 f   MSVCRT:utility.obj
 0001:000011d0       __scrt_is_nonwritable_in_current_image 00000001800021d0 f   MSVCRT:utility.obj
 0001:00001268       __scrt_release_startup_lock 0000000180002268 f   MSVCRT:utility.obj
 0001:0000128c       __scrt_uninitialize_crt    000000018000228c f   MSVCRT:utility.obj
 0001:000012b8       __scrt_get_dyn_tls_init_callback 00000001800022b8 f   MSVCRT:dyn_tls_init.obj
 0001:000012c0       __crt_debugger_hook        00000001800022c0 f   MSVCRT:utility_desktop.obj
 0001:000012c8       __scrt_fastfail            00000001800022c8 f   MSVCRT:utility_desktop.obj
 0001:00001410       _RTC_Initialize            0000000180002410 f   MSVCRT:initsect.obj
 0001:0000144c       _RTC_Terminate             000000018000244c f   MSVCRT:initsect.obj
 0001:00001488       _guard_check_icall_nop     0000000180002488 f i MSVCRT:guard_support.obj
 0001:0000148c       __isa_available_init       000000018000248c f   MSVCRT:cpu_disp.obj
 0001:00001758       _get_startup_argv_mode     0000000180002758 f   MSVCRT:argv_mode.obj
 0001:00001760       __scrt_is_ucrt_dll_in_use  0000000180002760 f   MSVCRT:ucrt_detection.obj
 0001:00001770       __C_specific_handler       0000000180002770 f   vcruntime:VCRUNTIME140.dll
 0001:00001776       __std_type_info_destroy_list 0000000180002776 f   vcruntime:VCRUNTIME140.dll
 0001:0000177c       memset                     000000018000277c f   vcruntime:VCRUNTIME140.dll
 0001:00001782       _initterm                  0000000180002782 f   ucrt:api-ms-win-crt-runtime-l1-1-0.dll
 0001:00001788       _initterm_e                0000000180002788 f   ucrt:api-ms-win-crt-runtime-l1-1-0.dll
 0001:0000178e       _seh_filter_dll            000000018000278e f   ucrt:api-ms-win-crt-runtime-l1-1-0.dll
 0001:00001794       _configure_narrow_argv     0000000180002794 f   ucrt:api-ms-win-crt-runtime-l1-1-0.dll
 0001:0000179a       _initialize_narrow_environment 000000018000279a f   ucrt:api-ms-win-crt-runtime-l1-1-0.dll
 0001:000017a0       _initialize_onexit_table   00000001800027a0 f   ucrt:api-ms-win-crt-runtime-l1-1-0.dll
 0001:000017a6       _execute_onexit_table      00000001800027a6 f   ucrt:api-ms-win-crt-runtime-l1-1-0.dll
 0001:000017ac       _cexit                     00000001800027ac f   ucrt:api-ms-win-crt-runtime-l1-1-0.dll
 0001:000017b4       __acrt_initialize          00000001800027b4 f   MSVCRT:ucrt_stubs.obj
 0001:000017b4       __acrt_thread_attach       00000001800027b4 f   MSVCRT:ucrt_stubs.obj
 0001:000017b4       __acrt_thread_detach       00000001800027b4 f   MSVCRT:ucrt_stubs.obj
 0001:000017b4       __acrt_uninitialize        00000001800027b4 f   MSVCRT:ucrt_stubs.obj
 0001:000017b4       __acrt_uninitialize_critical 00000001800027b4 f   MSVCRT:ucrt_stubs.obj
 0001:000017b4       __scrt_stub_for_acrt_initialize 00000001800027b4 f   MSVCRT:ucrt_stubs.obj
 0001:000017b4       __scrt_stub_for_acrt_thread_attach 00000001800027b4 f   MSVCRT:ucrt_stubs.obj
 0001:000017b4       __scrt_stub_for_acrt_thread_detach 00000001800027b4 f   MSVCRT:ucrt_stubs.obj
 0001:000017b4       __scrt_stub_for_acrt_uninitialize 00000001800027b4 f   MSVCRT:ucrt_stubs.obj
 0001:000017b4       __scrt_stub_for_acrt_uninitialize_critical 00000001800027b4 f   MSVCRT:ucrt_stubs.obj
 0001:000017b4       __vcrt_initialize          00000001800027b4 f   MSVCRT:ucrt_stubs.obj
 0001:000017b4       __vcrt_thread_attach       00000001800027b4 f   MSVCRT:ucrt_stubs.obj
 0001:000017b4       __vcrt_thread_detach       00000001800027b4 f   MSVCRT:ucrt_stubs.obj
 0001:000017b4       __vcrt_uninitialize        00000001800027b4 f   MSVCRT:ucrt_stubs.obj
 0001:000017b4       __vcrt_uninitialize_critical 00000001800027b4 f   MSVCRT:ucrt_stubs.obj
 0001:000017b8       __scrt_stub_for_is_c_termination_complete 00000001800027b8 f   MSVCRT:ucrt_stubs.obj
 0001:000017b8       _is_c_termination_complete 00000001800027b8 f   MSVCRT:ucrt_stubs.obj
 0001:000017bb       memcpy                     00000001800027bb f   vcruntime:VCRUNTIME140.dll
 0001:000017e0       _guard_dispatch_icall_nop  00000001800027e0 f   MSVCRT:guard_dispatch.obj
 0001:00001800       _guard_xfg_dispatch_icall_nop 0000000180002800 f   MSVCRT:guard_xfg_dispatch.obj
 0002:00000000       __imp_IsDebuggerPresent    0000000180003000     kernel32:KERNEL32.dll
 0002:00000008       __imp_InitializeSListHead  0000000180003008     kernel32:KERNEL32.dll
 0002:00000010       __imp_DisableThreadLibraryCalls 0000000180003010     kernel32:KERNEL32.dll
 0002:00000018       __imp_GetSystemTimeAsFileTime 0000000180003018     kernel32:KERNEL32.dll
 0002:00000020       __imp_GetCurrentThreadId   0000000180003020     kernel32:KERNEL32.dll
 0002:00000028       __imp_GetCurrentProcessId  0000000180003028     kernel32:KERNEL32.dll
 0002:00000030       __imp_RtlCaptureContext    0000000180003030     kernel32:KERNEL32.dll
 0002:00000038       __imp_RtlLookupFunctionEntry 0000000180003038     kernel32:KERNEL32.dll
 0002:00000040       __imp_RtlVirtualUnwind     0000000180003040     kernel32:KERNEL32.dll
 0002:00000048       __imp_UnhandledExceptionFilter 0000000180003048     kernel32:KERNEL32.dll
 0002:00000050       __imp_SetUnhandledExceptionFilter 0000000180003050     kernel32:KERNEL32.dll
 0002:00000058       __imp_GetCurrentProcess    0000000180003058     kernel32:KERNEL32.dll
 0002:00000060       __imp_TerminateProcess     0000000180003060     kernel32:KERNEL32.dll
 0002:00000068       __imp_IsProcessorFeaturePresent 0000000180003068     kernel32:KERNEL32.dll
 0002:00000070       __imp_QueryPerformanceCounter 0000000180003070     kernel32:KERNEL32.dll
 0002:00000078       \177KERNEL32_NULL_THUNK_DATA 0000000180003078     kernel32:KERNEL32.dll
 0002:00000080       __imp_memset               0000000180003080     vcruntime:VCRUNTIME140.dll
 0002:00000088       __imp___std_type_info_destroy_list 0000000180003088     vcruntime:VCRUNTIME140.dll
 0002:00000090       __imp___C_specific_handler 0000000180003090     vcruntime:VCRUNTIME140.dll
 0002:00000098       __imp_memcpy               0000000180003098     vcruntime:VCRUNTIME140.dll
 0002:000000a0       \177VCRUNTIME140_NULL_THUNK_DATA 00000001800030a0     vcruntime:VCRUNTIME140.dll
 0002:000000a8       __imp__cexit               00000001800030a8     ucrt:api-ms-win-crt-runtime-l1-1-0.dll
 0002:000000b0       __imp__execute_onexit_table 00000001800030b0     ucrt:api-ms-win-crt-runtime-l1-1-0.dll
 0002:000000b8       __imp__configure_narrow_argv 00000001800030b8     ucrt:api-ms-win-crt-runtime-l1-1-0.dll
 0002:000000c0       __imp__initialize_onexit_table 00000001800030c0     ucrt:api-ms-win-crt-runtime-l1-1-0.dll
 0002:000000c8       __imp__initterm            00000001800030c8     ucrt:api-ms-win-crt-runtime-l1-1-0.dll
 0002:000000d0       __imp__initterm_e          00000001800030d0     ucrt:api-ms-win-crt-runtime-l1-1-0.dll
 0002:000000d8       __imp__seh_filter_dll      00000001800030d8     ucrt:api-ms-win-crt-runtime-l1-1-0.dll
 0002:000000e0       __imp__initialize_narrow_environment 00000001800030e0     ucrt:api-ms-win-crt-runtime-l1-1-0.dll
 0002:000000e8       \177api-ms-win-crt-runtime-l1-1-0_NULL_THUNK_DATA 00000001800030e8     ucrt:api-ms-win-crt-runtime-l1-1-0.dll
 0002:000000f0       __imp___stdio_common_vsprintf 00000001800030f0     ucrt:api-ms-win-crt-stdio-l1-1-0.dll
 0002:000000f8       \177api-ms-win-crt-stdio-l1-1-0_NULL_THUNK_DATA 00000001800030f8     ucrt:api-ms-win-crt-stdio-l1-1-0.dll
 0002:00000100       __imp_JNU_ThrowInternalError 0000000180003100     java:java.dll
 0002:00000108       \177java_NULL_THUNK_DATA   0000000180003108     java:java.dll
 0002:00000110       __imp_JVM_ActiveProcessorCount 0000000180003110     jvm:jvm.dll
 0002:00000118       __imp_JVM_GetVmArguments   0000000180003118     jvm:jvm.dll
 0002:00000120       __imp_JVM_GetManagement    0000000180003120     jvm:jvm.dll
 0002:00000128       __imp_JVM_GetAllThreads    0000000180003128     jvm:jvm.dll
 0002:00000130       \177jvm_NULL_THUNK_DATA    0000000180003130     jvm:jvm.dll
 0002:00000138       __guard_check_icall_fptr   0000000180003138     MSVCRT:guard_support.obj
 0002:00000140       __guard_xfg_check_icall_fptr 0000000180003140     MSVCRT:guard_support.obj
 0002:00000148       __guard_dispatch_icall_fptr 0000000180003148     MSVCRT:guard_support.obj
 0002:00000150       __guard_xfg_dispatch_icall_fptr 0000000180003150     MSVCRT:guard_support.obj
 0002:00000158       __guard_xfg_table_dispatch_icall_fptr 0000000180003158     MSVCRT:guard_support.obj
 0002:00000160       __castguard_check_failure_os_handled_fptr 0000000180003160     MSVCRT:guard_support.obj
 0002:00000168       __guard_memcpy_fptr        0000000180003168     vcruntime:softmemtag.obj
 0002:00000170       __xc_a                     0000000180003170     MSVCRT:initializers.obj
 0002:00000178       __xc_z                     0000000180003178     MSVCRT:initializers.obj
 0002:00000180       __xi_a                     0000000180003180     MSVCRT:initializers.obj
 0002:00000188       __xi_z                     0000000180003188     MSVCRT:initializers.obj
 0002:00000190       __xp_a                     0000000180003190     MSVCRT:initializers.obj
 0002:00000198       __xp_z                     0000000180003198     MSVCRT:initializers.obj
 0002:000001a0       __xt_a                     00000001800031a0     MSVCRT:initializers.obj
 0002:000001a8       __xt_z                     00000001800031a8     MSVCRT:initializers.obj
 0002:000001b0       ??_C@_0BJ@KKOPABNE@Memory?5Manager?5not?5found@ 00000001800031b0     MemoryManagerImpl.obj
 0002:000001d0       ??_C@_0BG@EJKNNBCK@Memory?5Pool?5not?5found@ 00000001800031d0     MemoryPoolImpl.obj
 0002:000001e8       ??_C@_05KBEOJPB@?$CFd?4?$CFd@ 00000001800031e8     VMManagementImpl.obj
 0002:000001f0       ??_C@_01POHCFINO@Z@        00000001800031f0     VMManagementImpl.obj
 0002:000001f8       ??_C@_0BK@DJAAMHIC@compTimeMonitoringSupport@ 00000001800031f8     VMManagementImpl.obj
 0002:00000218       ??_C@_0CC@GDPMBOEP@threadContentionMonitoringSuppo@ 0000000180003218     VMManagementImpl.obj
 0002:00000240       ??_C@_0BM@GCPPCNJD@currentThreadCpuTimeSupport@ 0000000180003240     VMManagementImpl.obj
 0002:00000260       ??_C@_0BK@DMCEOMBH@otherThreadCpuTimeSupport@ 0000000180003260     VMManagementImpl.obj
 0002:00000280       ??_C@_0BK@EJFDBCBP@objectMonitorUsageSupport@ 0000000180003280     VMManagementImpl.obj
 0002:000002a0       ??_C@_0BJ@NIOHCHFH@synchronizerUsageSupport@ 00000001800032a0     VMManagementImpl.obj
 0002:000002c0       ??_C@_0BN@GDBJIKMK@threadAllocatedMemorySupport@ 00000001800032c0     VMManagementImpl.obj
 0002:000002e0       ??_C@_0CA@BBEOFMLC@remoteDiagnosticCommandsSupport@ 00000001800032e0     VMManagementImpl.obj
 0002:00000300       ??_C@_0BP@KJIDAONK@Unsupported?5Management?5version@ 0000000180003300     management.obj
 0002:00000320       _pDefaultRawDllMain        0000000180003320     MSVCRT:dll_dllmain.obj
 0002:00000320       _pRawDllMain               0000000180003320     MSVCRT:dll_dllmain.obj
 0002:00000340       __xmm@ffffffffffffffffffffffffffffffff 0000000180003340     MSVCRT:utility.obj
 0002:00000350       _load_config_used          0000000180003350     MSVCRT:loadcfg.obj
 0002:00000500       __volatile_metadata        0000000180003500     <linker-defined>
 0002:00000830       __rtc_iaa                  0000000180003830     MSVCRT:initsect.obj
 0002:00000838       __rtc_izz                  0000000180003838     MSVCRT:initsect.obj
 0002:00000840       __rtc_taa                  0000000180003840     MSVCRT:initsect.obj
 0002:00000848       __rtc_tzz                  0000000180003848     MSVCRT:initsect.obj
 0002:00001b4c       __IMPORT_DESCRIPTOR_java   0000000180004b4c     java:java.dll
 0002:00001b60       __IMPORT_DESCRIPTOR_jvm    0000000180004b60     jvm:jvm.dll
 0002:00001b74       __IMPORT_DESCRIPTOR_KERNEL32 0000000180004b74     kernel32:KERNEL32.dll
 0002:00001b88       __IMPORT_DESCRIPTOR_VCRUNTIME140 0000000180004b88     vcruntime:VCRUNTIME140.dll
 0002:00001b9c       __IMPORT_DESCRIPTOR_api-ms-win-crt-stdio-l1-1-0 0000000180004b9c     ucrt:api-ms-win-crt-stdio-l1-1-0.dll
 0002:00001bb0       __IMPORT_DESCRIPTOR_api-ms-win-crt-runtime-l1-1-0 0000000180004bb0     ucrt:api-ms-win-crt-runtime-l1-1-0.dll
 0002:00001bc4       __NULL_IMPORT_DESCRIPTOR   0000000180004bc4     java:java.dll
 0003:00000000       __security_cookie          0000000180006000     MSVCRT:gs_cookie.obj
 0003:00000040       __security_cookie_complement 0000000180006040     MSVCRT:gs_cookie.obj
 0003:00000048       __scrt_native_dllmain_reason 0000000180006048     MSVCRT:utility.obj
 0003:00000050       __isa_inverted             0000000180006050     MSVCRT:cpu_disp.obj
 0003:00000058       __isa_available            0000000180006058     MSVCRT:cpu_disp.obj
 0003:0000005c       __isa_enabled              000000018000605c     MSVCRT:cpu_disp.obj
 0003:00000060       __memset_fast_string_threshold 0000000180006060     MSVCRT:cpu_disp.obj
 0003:00000068       __memset_nt_threshold      0000000180006068     MSVCRT:cpu_disp.obj
 0003:00000070       __scrt_ucrt_dll_is_in_use  0000000180006070     MSVCRT:ucrt_stubs.obj
 0003:00000080       jmm_interface              0000000180006080     management.obj
 0003:00000088       jmm_version                0000000180006088     management.obj
 0003:00000610       ?__type_info_root_node@@3U__type_info_node@@A 0000000180006610     MSVCRT:tncleanup.obj
 0003:00000620       ?_OptionsStorage@?1??__local_stdio_scanf_options@@9@4_KA 0000000180006620     MSVCRT:default_local_stdio_options.obj
 0003:00000628       __scrt_current_native_startup_state 0000000180006628     MSVCRT:utility.obj
 0003:00000630       __scrt_native_startup_lock 0000000180006630     MSVCRT:utility.obj
 0003:00000670       __scrt_debugger_hook_flag  0000000180006670     MSVCRT:utility_desktop.obj
 0003:00000674       __avx10_version            0000000180006674     MSVCRT:cpu_disp.obj
 0003:00000678       __favor                    0000000180006678     MSVCRT:cpu_disp.obj
 0003:00000680       ?_OptionsStorage@?1??__local_stdio_printf_options@@9@9 0000000180006680     <common>
 0003:00000688       __dyn_tls_init_callback    0000000180006688     <common>

 entry point at        0001:00000cd0

 Static symbols

 0000:ffff6000       .debug$S                   0000000180000000     management.exp
 0000:ffff6000       .debug$S                   0000000180000000     vcruntime:VCRUNTIME140.dll
 0000:ffff6000       .debug$S                   0000000180000000     vcruntime:VCRUNTIME140.dll
 0000:ffff6000       .debug$S                   0000000180000000     vcruntime:VCRUNTIME140.dll
 0000:ffff6000       .debug$S                   0000000180000000     vcruntime:VCRUNTIME140.dll
 0000:ffff6000       .debug$S                   0000000180000000     vcruntime:VCRUNTIME140.dll
 0000:ffff6000       .debug$S                   0000000180000000     vcruntime:VCRUNTIME140.dll
 0000:ffff6000       .debug$S                   0000000180000000     ucrt:api-ms-win-crt-runtime-l1-1-0.dll
 0000:ffff6000       .debug$S                   0000000180000000     ucrt:api-ms-win-crt-runtime-l1-1-0.dll
 0000:ffff6000       .debug$S                   0000000180000000     ucrt:api-ms-win-crt-runtime-l1-1-0.dll
 0000:ffff6000       .debug$S                   0000000180000000     ucrt:api-ms-win-crt-runtime-l1-1-0.dll
 0000:ffff6000       .debug$S                   0000000180000000     ucrt:api-ms-win-crt-runtime-l1-1-0.dll
 0000:ffff6000       .debug$S                   0000000180000000     ucrt:api-ms-win-crt-runtime-l1-1-0.dll
 0000:ffff6000       .debug$S                   0000000180000000     ucrt:api-ms-win-crt-runtime-l1-1-0.dll
 0000:ffff6000       .debug$S                   0000000180000000     ucrt:api-ms-win-crt-runtime-l1-1-0.dll
 0000:ffff6000       .debug$S                   0000000180000000     ucrt:api-ms-win-crt-runtime-l1-1-0.dll
 0000:ffff6000       .debug$S                   0000000180000000     ucrt:api-ms-win-crt-runtime-l1-1-0.dll
 0000:ffff6000       .debug$S                   0000000180000000     ucrt:api-ms-win-crt-runtime-l1-1-0.dll
 0000:ffff6000       .debug$S                   0000000180000000     ucrt:api-ms-win-crt-runtime-l1-1-0.dll
 0000:ffff6000       .debug$S                   0000000180000000     ucrt:api-ms-win-crt-stdio-l1-1-0.dll
 0000:ffff6000       .debug$S                   0000000180000000     kernel32:KERNEL32.dll
 0000:ffff6000       .debug$S                   0000000180000000     kernel32:KERNEL32.dll
 0000:ffff6000       .debug$S                   0000000180000000     kernel32:KERNEL32.dll
 0000:ffff6000       .debug$S                   0000000180000000     kernel32:KERNEL32.dll
 0000:ffff6000       .debug$S                   0000000180000000     kernel32:KERNEL32.dll
 0000:ffff6000       .debug$S                   0000000180000000     kernel32:KERNEL32.dll
 0000:ffff6000       .debug$S                   0000000180000000     kernel32:KERNEL32.dll
 0000:ffff6000       .debug$S                   0000000180000000     kernel32:KERNEL32.dll
 0000:ffff6000       .debug$S                   0000000180000000     kernel32:KERNEL32.dll
 0000:ffff6000       .debug$S                   0000000180000000     kernel32:KERNEL32.dll
 0000:ffff6000       .debug$S                   0000000180000000     kernel32:KERNEL32.dll
 0000:ffff6000       .debug$S                   0000000180000000     kernel32:KERNEL32.dll
 0000:ffff6000       .debug$S                   0000000180000000     kernel32:KERNEL32.dll
 0000:ffff6000       .debug$S                   0000000180000000     kernel32:KERNEL32.dll
 0000:ffff6000       .debug$S                   0000000180000000     kernel32:KERNEL32.dll
 0000:ffff6000       .debug$S                   0000000180000000     kernel32:KERNEL32.dll
 0000:ffff6000       .debug$S                   0000000180000000     kernel32:KERNEL32.dll
 0000:ffff6000       .debug$S                   0000000180000000     jvm:jvm.dll
 0000:ffff6000       .debug$S                   0000000180000000     jvm:jvm.dll
 0000:ffff6000       .debug$S                   0000000180000000     jvm:jvm.dll
 0000:ffff6000       .debug$S                   0000000180000000     jvm:jvm.dll
 0000:ffff6000       .debug$S                   0000000180000000     java:java.dll
 0001:000007d8       setStaticBooleanField      00000001800017d8 f   VMManagementImpl.obj
 0001:00000990       $$000000                   0000000180001990     MSVCRT:amdsecgs.obj
 0001:000009c0       ?dllmain_crt_dispatch@@YAHQEAUHINSTANCE__@@KQEAX@Z 00000001800019c0 f   MSVCRT:dll_dllmain.obj
 0001:00000a10       ?dllmain_crt_process_attach@@YAHQEAUHINSTANCE__@@QEAX@Z 0000000180001a10 f   MSVCRT:dll_dllmain.obj
 0001:00000b28       ?dllmain_crt_process_detach@@YAH_N@Z 0000000180001b28 f   MSVCRT:dll_dllmain.obj
 0001:00000ba8       ?dllmain_dispatch@@YAHQEAUHINSTANCE__@@KQEAX@Z 0000000180001ba8 f   MSVCRT:dll_dllmain.obj
 0001:00000e18       capture_previous_context   0000000180001e18 f   MSVCRT:gs_report.obj
 0001:000017d0       $$000000                   00000001800027d0     MSVCRT:guard_dispatch.obj
 0001:000017f0       $$000000                   00000001800027f0     MSVCRT:guard_xfg_dispatch.obj
 0001:00001806       ?fin$0@?0??dllmain_crt_process_attach@@YAHQEAUHINSTANCE__@@QEAX@Z@4HA 0000000180002806 f   MSVCRT:dll_dllmain.obj
 0001:0000181d       ?fin$0@?0??dllmain_crt_process_detach@@YAH_N@Z@4HA 000000018000281d f   MSVCRT:dll_dllmain.obj
 0001:00001836       ?fin$1@?0??dllmain_crt_process_detach@@YAH_N@Z@4HA 0000000180002836 f   MSVCRT:dll_dllmain.obj
 0001:0000184a       ?filt$0@?0??dllmain_dispatch@@YAHQEAUHINSTANCE__@@KQEAX@Z@4HA 000000018000284a f   MSVCRT:dll_dllmain.obj
 0001:00001880       __scrt_is_nonwritable_in_current_image$filt$0 0000000180002880 f   MSVCRT:utility.obj
 0002:00000328       GS_ExceptionPointers       0000000180003328     MSVCRT:gs_report.obj
 0002:00000850       $unwind$Java_sun_management_MemoryManagerImpl_getMemoryPools0 0000000180003850     MemoryManagerImpl.obj
 0002:00000850       $unwind$Java_sun_management_MemoryPoolImpl_getMemoryManagers0 0000000180003850     MemoryPoolImpl.obj
 0002:00000850       $unwind$Java_sun_management_MemoryPoolImpl_getPeakUsage0 0000000180003850     MemoryPoolImpl.obj
 0002:00000850       $unwind$Java_sun_management_MemoryPoolImpl_getUsage0 0000000180003850     MemoryPoolImpl.obj
 0002:00000850       $unwind$Java_sun_management_VMManagementImpl_initOptionalSupportFields 0000000180003850     VMManagementImpl.obj
 0002:00000850       $unwind$_RTC_Initialize    0000000180003850     MSVCRT:initsect.obj
 0002:00000850       $unwind$_RTC_Terminate     0000000180003850     MSVCRT:initsect.obj
 0002:0000085c       $unwind$Java_sun_management_MemoryPoolImpl_setCollectionThreshold0 000000018000385c     MemoryPoolImpl.obj
 0002:0000085c       $unwind$Java_sun_management_MemoryPoolImpl_setUsageThreshold0 000000018000385c     MemoryPoolImpl.obj
 0002:0000085c       $unwind$setStaticBooleanField 000000018000385c     VMManagementImpl.obj
 0002:0000085c       $unwind$_DllMainCRTStartup 000000018000385c     MSVCRT:dll_dllmain.obj
 0002:0000086c       $unwind$snprintf           000000018000386c     VMManagementImpl.obj
 0002:0000087c       $unwind$Java_sun_management_VMManagementImpl_getVersion0 000000018000387c     VMManagementImpl.obj
 0002:0000088c       $unwind$JNI_OnLoad         000000018000388c     management.obj
 0002:0000088c       $unwind$__scrt_initialize_default_local_stdio_options 000000018000388c     MSVCRT:default_local_stdio_options.obj
 0002:0000088c       $unwind$?dllmain_crt_dispatch@@YAHQEAUHINSTANCE__@@KQEAX@Z 000000018000388c     MSVCRT:dll_dllmain.obj
 0002:0000088c       $unwind$DllMain            000000018000388c     MSVCRT:dll_dllmain_stub.obj
 0002:0000088c       $unwind$__GSHandlerCheck   000000018000388c     MSVCRT:gshandler.obj
 0002:0000088c       $unwind$__scrt_acquire_startup_lock 000000018000388c     MSVCRT:utility.obj
 0002:0000088c       $unwind$__scrt_dllmain_after_initialize_c 000000018000388c     MSVCRT:utility.obj
 0002:0000088c       $unwind$__scrt_dllmain_before_initialize_c 000000018000388c     MSVCRT:utility.obj
 0002:0000088c       $unwind$__scrt_dllmain_crt_thread_attach 000000018000388c     MSVCRT:utility.obj
 0002:0000088c       $unwind$__scrt_dllmain_crt_thread_detach 000000018000388c     MSVCRT:utility.obj
 0002:0000088c       $unwind$__scrt_dllmain_uninitialize_c 000000018000388c     MSVCRT:utility.obj
 0002:0000088c       $unwind$__scrt_dllmain_uninitialize_critical 000000018000388c     MSVCRT:utility.obj
 0002:0000088c       $unwind$__scrt_initialize_crt 000000018000388c     MSVCRT:utility.obj
 0002:00000894       $unwind$__GSHandlerCheckCommon 0000000180003894     MSVCRT:gshandler.obj
 0002:000008a0       $xdatasym                  00000001800038a0     MSVCRT:amdsecgs.obj
 0002:000008a4       $unwind$?dllmain_crt_process_attach@@YAHQEAUHINSTANCE__@@QEAX@Z 00000001800038a4     MSVCRT:dll_dllmain.obj
 0002:000008e0       $unwind$?fin$0@?0??dllmain_crt_process_attach@@YAHQEAUHINSTANCE__@@QEAX@Z@4HA 00000001800038e0     MSVCRT:dll_dllmain.obj
 0002:000008e0       $unwind$?fin$0@?0??dllmain_crt_process_detach@@YAH_N@Z@4HA 00000001800038e0     MSVCRT:dll_dllmain.obj
 0002:000008e0       $unwind$?fin$1@?0??dllmain_crt_process_detach@@YAH_N@Z@4HA 00000001800038e0     MSVCRT:dll_dllmain.obj
 0002:000008e8       $unwind$?dllmain_crt_process_detach@@YAH_N@Z 00000001800038e8     MSVCRT:dll_dllmain.obj
 0002:0000093c       $unwind$?dllmain_dispatch@@YAHQEAUHINSTANCE__@@KQEAX@Z 000000018000393c     MSVCRT:dll_dllmain.obj
 0002:00000964       $unwind$?filt$0@?0??dllmain_dispatch@@YAHQEAUHINSTANCE__@@KQEAX@Z@4HA 0000000180003964     MSVCRT:dll_dllmain.obj
 0002:0000096c       $unwind$__report_gsfailure 000000018000396c     MSVCRT:gs_report.obj
 0002:00000974       $unwind$capture_previous_context 0000000180003974     MSVCRT:gs_report.obj
 0002:00000980       $unwind$__raise_securityfailure 0000000180003980     MSVCRT:gs_report.obj
 0002:00000980       $unwind$__scrt_initialize_onexit_tables 0000000180003980     MSVCRT:utility.obj
 0002:00000980       $unwind$__scrt_release_startup_lock 0000000180003980     MSVCRT:utility.obj
 0002:00000980       $unwind$__scrt_uninitialize_crt 0000000180003980     MSVCRT:utility.obj
 0002:00000988       $unwind$__security_init_cookie 0000000180003988     MSVCRT:gs_support.obj
 0002:00000994       $unwind$__scrt_is_nonwritable_in_current_image 0000000180003994     MSVCRT:utility.obj
 0002:000009b4       $unwind$__scrt_is_nonwritable_in_current_image$filt$0 00000001800039b4     MSVCRT:utility.obj
 0002:000009bc       $unwind$__scrt_dllmain_exception_filter 00000001800039bc     MSVCRT:utility.obj
 0002:000009d0       $unwind$__scrt_fastfail    00000001800039d0     MSVCRT:utility_desktop.obj
 0002:000009e0       $unwind$__isa_available_init 00000001800039e0     MSVCRT:cpu_disp.obj
 0002:000009f8       $xdatasym                  00000001800039f8     MSVCRT:guard_dispatch.obj
 0002:00000a00       $xdatasym                  0000000180003a00     MSVCRT:guard_xfg_dispatch.obj
 0002:00000a10       .edata                     0000000180003a10     management.exp
 0002:00000a38       rgpv                       0000000180003a38     management.exp
 0002:00000b44       rgszName                   0000000180003b44     management.exp
 0002:00000c50       rgwOrd                     0000000180003c50     management.exp
 0002:00000cd6       szName                     0000000180003cd6     management.exp
 0002:00000ce5       $N00001                    0000000180003ce5     management.exp
 0002:00000cf0       $N00002                    0000000180003cf0     management.exp
 0002:00000d25       $N00003                    0000000180003d25     management.exp
 0002:00000d61       $N00004                    0000000180003d61     management.exp
 0002:00000d9c       $N00005                    0000000180003d9c     management.exp
 0002:00000dd5       $N00006                    0000000180003dd5     management.exp
 0002:00000e0f       $N00007                    0000000180003e0f     management.exp
 0002:00000e41       $N00008                    0000000180003e41     management.exp
 0002:00000e70       $N00009                    0000000180003e70     management.exp
 0002:00000e9f       $N00010                    0000000180003e9f     management.exp
 0002:00000ecb       $N00011                    0000000180003ecb     management.exp
 0002:00000f01       $N00012                    0000000180003f01     management.exp
 0002:00000f38       $N00013                    0000000180003f38     management.exp
 0002:00000f6e       $N00014                    0000000180003f6e     management.exp
 0002:00000f9f       $N00015                    0000000180003f9f     management.exp
 0002:00000fcc       $N00016                    0000000180003fcc     management.exp
 0002:00000fff       $N00017                    0000000180003fff     management.exp
 0002:0000103a       $N00018                    000000018000403a     management.exp
 0002:00001075       $N00019                    0000000180004075     management.exp
 0002:000010ab       $N00020                    00000001800040ab     management.exp
 0002:000010e1       $N00021                    00000001800040e1     management.exp
 0002:0000110d       $N00022                    000000018000410d     management.exp
 0002:00001143       $N00023                    0000000180004143     management.exp
 0002:00001180       $N00024                    0000000180004180     management.exp
 0002:000011b9       $N00025                    00000001800041b9     management.exp
 0002:000011f2       $N00026                    00000001800041f2     management.exp
 0002:00001220       $N00027                    0000000180004220     management.exp
 0002:00001256       $N00028                    0000000180004256     management.exp
 0002:0000128c       $N00029                    000000018000428c     management.exp
 0002:000012c1       $N00030                    00000001800042c1     management.exp
 0002:000012f6       $N00031                    00000001800042f6     management.exp
 0002:00001320       $N00032                    0000000180004320     management.exp
 0002:0000135d       $N00033                    000000018000435d     management.exp
 0002:00001392       $N00034                    0000000180004392     management.exp
 0002:000013c7       $N00035                    00000001800043c7     management.exp
 0002:00001407       $N00036                    0000000180004407     management.exp
 0002:0000144c       $N00037                    000000018000444c     management.exp
 0002:00001484       $N00038                    0000000180004484     management.exp
 0002:000014c0       $N00039                    00000001800044c0     management.exp
 0002:00001500       $N00040                    0000000180004500     management.exp
 0002:00001539       $N00041                    0000000180004539     management.exp
 0002:00001577       $N00042                    0000000180004577     management.exp
 0002:000015b1       $N00043                    00000001800045b1     management.exp
 0002:000015ef       $N00044                    00000001800045ef     management.exp
 0002:00001627       $N00045                    0000000180004627     management.exp
 0002:0000165f       $N00046                    000000018000465f     management.exp
 0002:00001696       $N00047                    0000000180004696     management.exp
 0002:000016ce       $N00048                    00000001800046ce     management.exp
 0002:00001700       $N00049                    0000000180004700     management.exp
 0002:00001737       $N00050                    0000000180004737     management.exp
 0002:00001771       $N00051                    0000000180004771     management.exp
 0002:000017a5       $N00052                    00000001800047a5     management.exp
 0002:000017ec       $N00053                    00000001800047ec     management.exp
 0002:00001824       $N00054                    0000000180004824     management.exp
 0002:0000185d       $N00055                    000000018000485d     management.exp
 0002:00001898       $N00056                    0000000180004898     management.exp
 0002:000018d1       $N00057                    00000001800048d1     management.exp
 0002:0000190c       $N00058                    000000018000490c     management.exp
 0002:00001946       $N00059                    0000000180004946     management.exp
 0002:00001976       $N00060                    0000000180004976     management.exp
 0002:000019ab       $N00061                    00000001800049ab     management.exp
 0002:000019dd       $N00062                    00000001800049dd     management.exp
 0002:00001a0e       $N00063                    0000000180004a0e     management.exp
 0002:00001a43       $N00064                    0000000180004a43     management.exp
 0002:00001a82       $N00065                    0000000180004a82     management.exp
 0002:00001ac6       $N00066                    0000000180004ac6     management.exp
 0002:00001b0f       $N00067                    0000000180004b0f     management.exp
 0002:00001d2a       .idata$6                   0000000180004d2a     java:java.dll
 0002:00001d8e       .idata$6                   0000000180004d8e     jvm:jvm.dll
 0002:00001efc       .idata$6                   0000000180004efc     kernel32:KERNEL32.dll
 0002:00001f4c       .idata$6                   0000000180004f4c     vcruntime:VCRUNTIME140.dll
 0002:0000201e       .idata$6                   000000018000501e     ucrt:api-ms-win-crt-stdio-l1-1-0.dll
 0002:0000203e       .idata$6                   000000018000503e     ucrt:api-ms-win-crt-runtime-l1-1-0.dll
 0003:00000090       jvm                        0000000180006090     management.obj
 0003:00000098       ?__proc_attached@@3HA      0000000180006098     MSVCRT:dll_dllmain.obj
 0003:000000a0       GS_ExceptionRecord         00000001800060a0     MSVCRT:gs_report.obj
 0003:00000140       GS_ContextRecord           0000000180006140     MSVCRT:gs_report.obj
 0003:00000638       ?is_initialized_as_dll@@3_NA 0000000180006638     MSVCRT:utility.obj
 0003:00000639       ?module_local_atexit_table_initialized@@3_NA 0000000180006639     MSVCRT:utility.obj
 0003:00000640       ?module_local_atexit_table@@3U_onexit_table_t@@A 0000000180006640     MSVCRT:utility.obj
 0003:00000658       ?module_local_at_quick_exit_table@@3U_onexit_table_t@@A 0000000180006658     MSVCRT:utility.obj
 0005:00000060       $R000000                   0000000180008060     management.dll.res
